:100000000080001041000000850000008500000015
:10001000850000008500000085000000267DFFEFC0
:10002000000000000000000000000000850000004B
:100030008500000000000000850000007D01000038
:1000400008B500F021F80A4A0A4B0B4903E052F8C0
:10005000040B43F8040B8B42F9D3084B08490022E8
:1000600001E043F8042B8B42FBD300F08FF8FEE74E
:100070003402000000000010040000100400001012
:1000800004000010FEE70000344B2022C3F8A0213A
:100090001A46D2F8A011314B11F0400FF9D00322CB
:1000A000C3F804210022C3F8A821C3F8AC212C4ACC
:1000B0000120C3F80C01AA21C3F884205522C3F8FB
:1000C0008C10C3F88C20C3F88000C3F88C10C3F8E0
:1000D0008C20D3F88810214A11F0806FF9D00323C7
:1000E000C2F88030A733C2F88C305523C2F88C3068
:1000F000D2F88810194B11F0407FF9D02322C3F8B1
:10010000A420AA2132320120C3F8AC10C3F8AC20DD
:10011000C3F8A000C3F8AC10C3F8AC20D3F8A81003
:100120000E4A11F4806FF9D00323C2F8A030A73330
:10013000C2F8AC305523C2F8AC30D2F8A810074B47
:1001400011F4407FF9D0074AC3F8C4200022C3F855
:10015000C82143F23A021A60704700BF00C00F4046
:1001600063000500DE872804034B1A681968891AA2
:100170007729FBD9704700BF04000010024B1A68B2
:1001800001321A60704700BF04000010254BF7B51C
:100190001A684FF47A73B2FBF3F222F07F42224BDB
:1001A000013A5A60214AF82182F8231000229A600D
:1001B0001F4C07321A6023684FF4802743F48023D2
:1001C000236023683A4643F48013236023684FF486
:1001D000801643F40013236023684FF4001543F0A6
:1001E00000532360E2610092FFF7BEFFA761A661A2
:1001F000FFF7BAFFE661A561FFF7B6FF4FF00053C6
:10020000E561A3610193FFF7AFFF019BE361A56186
:10021000FFF7AAFFE561A661FFF7A6FFE661009A76
:10022000E0E700BF0000001010E000E000ED00E09B
:0402300020C00920C1
:0402340000E1F505EB
:0400000300000041B8
:00000001FF
